:020000040000FA
:1000000008030020F9000000FD000000D5000000FA
:1000100000000000000000000000000000000000E0
:1000200000000000000000000000000001010000CE
:1000300000000000000000000301000005010000B6
:100040000701000007010000ED050000090600009F
:100050000701000007010000070100000701000080
:10006000BD090000D90900000701000007010000D8
:10007000F50900000701000007010000070100006A
:100080000701000007010000070100000701000050
:100090000701000007010000070100000701000040
:1000A0000701000007010000070100000701000030
:1000B0000701000007010000070100000701000020
:1000C0000348854600F068F800480047D90F000053
:1000D0000803002004207146084202D0EFF3098093
:1000E00001E0EFF308807146004A10475506000012
:1000F000401EFDD27047000003480047FEE7FEE7C0
:10010000FEE7FEE7FEE7FEE7C100000030B50B4664
:10011000014600202022012409E00D46D5409D42E1
:1001200005D31D469540491B254695404019154667
:10013000521E002DF1DC30BDF0B51FB40646002084
:1001400082B005464024019100901BE001992246AF
:100150000F46304600F042F8049A059B801A9941F8
:1001600010D310461946224600F028F8361A8F415F
:100170000197224601200021009F00F01FF8381847
:100180004D4100902046641E0028DFDC019B009852
:100190002946324607B0F0BD064C0125064E05E063
:1001A000E36807CC2B430C3C98471034B442F7D398
:1001B000FFF78AFF88160000A816000010B5202A55
:1001C00004DB0146203A9140002010BD91402023DD
:1001D0009C1A0346E3401943904010BD10B5202AF5
:1001E00004DB0846203AD040002110BD0B46D34026
:1001F000D0402024A21A91400843194610BD0000A7
:100200000248016AC20111430162704700020050B6
:10021000C10F8A00044951184A68C306DB0E012049
:10022000984002434A60704700020050F3B58BB01B
:100230000C46FFF7E5FF0B9800287448016813D0BF
:10024000042211430160102000F0BCF90120C00419
:1002500009906F480090042008906E486E4920185D
:1002600088420ED800251DE089088900491C0160DC
:10027000012000F0A7F900200990684800900220B2
:10028000EAE76748664920184942884202D80125B2
:10029000640007E0634863492018494288427DD2E0
:1002A0000325A4000026F643089F22E03946009863
:1002B000FFF72CFF5C49844641185C48814217D205
:1002C000554B02225B1C534861465143401C0818A1
:1002D000984209D8A14201D9081B00E0601AB04237
:1002E00002D2060004920CD05148521C8242EAD934
:1002F0007F1C212FDAD900200696C0430190089E6A
:1003000054E00999A803084301217A028902511A8D
:1003100008430499891E08433C490862042000F000
:1003200051F9691C79430098FFF7F0FE049948439E
:100330000DB0F0BD31460098FFF7E8FE3A4942188B
:100340003A498A4231D20221324B02464A435B1C6F
:10035000D7185B429F4224D8A24201D9121B00E069
:10036000A21A019B9A421CD20192069B0F469A4206
:1003700017D10999A8030843012172028902511A71
:100380000843B91E084321490862042000F01AF905
:10039000691C71430098FFF7B9FE00E008E078435C
:1003A000C6E7234A491C9142CED9761C212EC1D9D9
:1003B0000B9800280FD01F4914480162042000F058
:1003C00001F91DA0006803901048016A0013014262
:1003D00003D00020ACE71949EEE7080301D50C482B
:1003E00000E00E488A03A3D40A04920F03AB9B5C7F
:1003F000CA058904D20DC90E891C8008921C594374
:100400005043FFF783FE800092E700000002005097
:1004100000805101FF1E0AFAFFE0F505001BB7003E
:10042000800F05FDC08782FEFF95E7FFBF77CC00F8
:1004300001020000184408000102020416400000F6
:10044000044982070A6801D09208920002430A60B8
:10045000704700000002005010B500F00BFA014890
:10046000006810BD08000020044800688007800F65
:10047000012801D000207047014870470002005059
:10048000001BB700044800688007800F022801D0D5
:10049000002070470148704700020050001BB70061
:1004A00008B511A0006800901048016A00130142CD
:1004B00001D0002008BD080301D50D4800E00D481B
:1004C0008A03F7D40A04920F6B469B5CCA05890421
:1004D000D20DC90E891C8008921C59435043FFF766
:1004E00015FE800008BD0000010202040002005059
:1004F00000805101001BB70008B511A000680090F2
:100500001048016A0013014201D0002008BD080311
:1005100001D50D4800E00D488A03F7D40A04920F74
:100520006B469B5CCA058904D20DC90E891C8008E4
:10053000921C59435043FFF7E9FD800008BD0000BD
:10054000010202040002005000805101001BB700AC
:1005500010B5074A93691B091B010B43936111698D
:10056000C908C9000143116100F084F910BD000001
:100570000002005070B5430E1B070DD043009B0FC7
:100580000F4C9B001C192368C5002D0FC601F60EE9
:10059000B540AB430B432360840A2106090E0DD0FE
:1005A0000103074B890F89000833CB1819688005B0
:1005B000E4B2C00E8440A1431143196070BD000035
:1005C0001002005010B50749074A05E00B46491EC6
:1005D000002B01DC002010BDD4680346A343F5D1F5
:1005E000012010BD80F520000002005004490420C5
:1005F000086204484068002800D0004770470000A7
:10060000C0400050580000200449042008620448FB
:100610000068002800D000477047000040410050AB
:1006200058000020F0B500230125944603272A46F0
:100630009A400A4209D006685C003A46A2409643B6
:10064000224664469440264306605B1C082BEED38A
:10065000F0BD0000044603A000F044FA204600F07C
:1006600017FEFEE7496E2048617264204661756C92
:10067000742048616E646C65720A00008307FF2273
:10068000DB0E9A408907090E994000280BDA000713
:10069000000F0838830808489B001818C369934363
:1006A0000B43C3617047830804489B001B181868FC
:1006B000904308431860704700ED00E000E400E05C
:1006C0008168082291438160704710B5029C202BFD
:1006D00000D10023DB000B4313430360012292048B
:1006E000914201D110218160214600F001F810BD36
:1006F00070B5064619480D4641698906890F21D013
:1007000040698006800F022823D0FFF7A5FE04462B
:10071000A54200D90546002D1ED029462046FFF7E8
:10072000F5FC401C4008401EFF2800D9FF207168DE
:10073000090A09020143716041002046891CFFF744
:10074000E5FC70BDFFF790FE0400E1D1FFF79AFED3
:10075000DDE7FFF7D1FEDAE7002070BD00020050B0
:10076000F8B55921304C1622882021602260206083
:100770002368002BF9D02D4D04202860FFF760FE80
:100780000820FFF75DFE1020FFF71CFF28690721F6
:1007900008432861A86900090001A8612449A8024A
:1007A000FFF744FD01210220FFF7D2FE2148FFF7A9
:1007B0002FFD214E3046FFF72BFDB32212040821F6
:1007C0003046FFF7D7FE1D48FFF722FD1C48FFF714
:1007D0001FFD00F04FF81BA000680090286A291345
:1007E00001400025002901D02A4616E0010301D569
:1007F000154A00E0154A81030FD40104890F6B46A6
:100800005E5CC3058004C10EDB0D891C90089B1C37
:1008100071435843FFF77AFC82000D4EB260FFF738
:100820001BFEF0602560F8BD000100500002005082
:1008300000E1F505103D80A71CFE23A61400C0A70B
:100840001500E0A70102020400805101001BB7005F
:100850001400002006498A691202FCD408600A28A4
:1008600004D188690002FCD40D20086070470000A4
:1008700000000540F8B520A00068204E0090316AC5
:1008800030131F4C1F4F014201D0002016E0080317
:1008900001D5204600E038468A030FD40A04920F9F
:1008A0006B469B5CCA058904D20DC90E891C800861
:1008B000921C59435043FFF729FC8000124D2860D9
:1008C00031694907490F12D0022902D0032910D0FB
:1008D0002046B1690907090F491CFFF717FC0B49AE
:1008E00068604A108018FFF711FCA860F8BD384610
:1008F000EFE70748EDE700000102020400020050A4
:1009000000805101001BB7000400002040420F008E
:10091000102700000F4A10499042486901D1000A8F
:1009200000E0000B4007400F06D001280ED002283F
:100930000ED00A480068704708688007800F0128B9
:1009400002D00120C0037047054870470548704732
:100950000548EFE7000001400002005000000020C1
:10096000001BB7001027000008000020F8B5134650
:100970000F460646FFF7CEFF044600254008984282
:1009800001D2022010E0012149068C4202D3032546
:10099000A40805E0012109068C4201D30125044683
:1009A00019462046FFF7B2FB2F43376070606D1C7D
:1009B000684301462046FFF7A9FBF8BD0449012022
:1009C000886004480068002800D000477047000095
:1009D00000000140600000200449012088600448B4
:1009E0004068002800D00047704700002000014008
:1009F0006000002070B51849CD690022EB05174C46
:100A00001748002B0BDB0DE00378202B04D20E6877
:100A1000E6545B1C037002E002700B682370CB6924
:100A2000DB07F1D1AB0515D543888488A34211D2E9
:100A3000002C0FD0094D2035ED5C5B1C45709BB23E
:100A400043800D60A34205D3828042804868022221
:100A50009043486070BD000000000540B0000020D9
:100A60006800002070B51B4E0D46044671690020D9
:100A700089010322890F2063E260A06000291FD052
:100A800001291FD0022901D313480068B169090563
:100A9000090F491CFFF73AFB0646002D19D06808DC
:100AA00080192946FFF732FB0C49801E88420CD979
:100AB000E80080192946FFF729FB0009801E07E09E
:100AC0000748E3E7FFF7ECFCE0E7032109070843E9
:100AD000606270BD0002005000000020FFFF0000B7
:100AE000001BB7000FB410B503A9044B044A0298C9
:100AF00000F094F810BC08BC04B018476D0F00005B
:100B00001000002002E008C8121F08C1002AFAD114
:100B100070477047002001E001C1121F002AFBD17D
:100B2000704710B504460089FFF7E2FA61680120BA
:100B300008606089FFF7DCFA61680020086020899E
:100B4000FFF7D6FA10BD70B50446006801250560B0
:100B50002089FFF7CDFA606805602089FFF7C8FAA1
:100B6000206800686168C5B2002008602089FFF72E
:100B7000BFFA284670BDF8B500260446354637460C
:100B800076002089FFF7B4FA6168012008602089A7
:100B9000FFF7AEFA206800683043C6B260680760AD
:100BA0002089FFF7A5FA6D1CEDB2082DE8D3304679
:100BB000F8BD70B5044621680120086061680860CE
:100BC0002089FFF795FA2068002505602089FFF746
:100BD0008FFA606805602089FFF78AFA70BD70B5EA
:100BE00004462168002008606068012505602089AE
:100BF000FFF77EFA2068056070BD70B506460D46A9
:100C000000243168E80908603046FFF78AFF68066B
:100C1000641C050EE4B2082CF3D370BDFFB58FB091
:100C20000F460446002606E025280AD0129A11999C
:100C30009047641C761C20780028F5D1304613B00C
:100C4000F0BD00250121A14A009500E00543641C88
:100C500023780846203B98401042F7D120782E2870
:100C600015D1042005436078641C2A280AD101CFDD
:100C7000641C00900BE000990A225143303940185F
:100C8000641C00902078014630390929F3D9207876
:100C90006C280ED004DC4C2813D06A2812D104E052
:100CA00074280ED07A280DD10BE0012040050543B1
:100CB00007E00121090562780D43824201D16D18D8
:100CC000641C641C2078864669284AD008DC002809
:100CD000B4D058286DD0632810D0642808D140E0E3
:100CE00070286BD0732812D0752860D0782860D017
:100CF000129A704611999047761CE5E0387869465B
:100D000008720020487202A80190012003E03868B0
:100D100001900020C0433F1D69070CD5002500E06D
:100D20006D1C00998D420FDA8542F9DB0199495D0E
:100D30000029F5D108E0002500E06D1C8542FCDBB0
:100D40000199495D0029F8D1761907E001980199C8
:100D50000078491C0191129A119990476D1EF5D2A5
:100D6000B2E00A20029000216802400F039102289D
:100D70000CD001CFC117844600290DDA624608461F
:100D800052420021814194462D2008E0FF1DFF08BA
:100D9000FF0003CF8446EFE7280504D52B206A46E1
:100DA000107401203CE0E8073AD02020F7E70A2041
:100DB00000E0102000210391029007E01020029033
:100DC0000021042005430820039100906802400F91
:100DD000022810D001CF0021844600200D90280762
:100DE0001FD5704670280CD0029A1020039B4240F9
:100DF0001A430CD015E0FF1DFF08FF0003CF844607
:100E0000EBE740206A46107401200D900CE060462C
:100E1000084306D030206A46107470465074022091
:100E20000D907046582804D029A001900DA80E906E
:100E30000DE02CA0F9E76046039B029AFFF77CF9CE
:100E4000019B84469B5C0E9A521E0E921370604664
:100E50000843F0D10E9805A9081A203001906807C0
:100E600001D5009801E0012000900199884203DD3E
:100E700001460198081A00E000200025009006E0D5
:100E800004A8129A405D119990476D1C761C0D982C
:100E90008542F5DB04E0129A302011999047761CC8
:100EA0000099481E00900029F5DC08E00E980E9984
:100EB0000078491C0E91129A11999047761C01995D
:100EC000481E01900029F1DC641CB4E609280100E9
:100ED00030313233343536373839616263646566B0
:100EE0000000000030313233343536373839414272
:100EF00043444546000000000A48016A01221143AC
:100F0000016205200007416B074A11404163416BB4
:100F100008221143416305484168120411434160AE
:100F20007047000000000E40F7F7FFF74040005008
:100F300004488169002902D00021816170470121A4
:100F4000FBE700004042005010B505200007816B10
:100F50008163012240210348FFF764FB024900201E
:100F6000886110BD804000504042005000B50346EB
:100F7000FFF770FC184600BD1CB503200521084C86
:100F800002460191009004232146064800F0DCF956
:100F90000449224608460C3000F0CEF91CBD000082
:100FA00003000300F0000020F8B50E460093C1B224
:100FB0001346069D079C3246064800F0F5F90028C6
:100FC00003D0002D00D0A847F8BD002CFCD0A047CE
:100FD000F8BD0000F0000020FFF7C2FBFFF7CCFFD8
:100FE00000F0F6F8012000F027F8FFF785FF00F089
:100FF000DBF800F051FAFF200949F53000F022FA41
:1010000008A0FFF76FFDFFF79FFF7C26094DFFF754
:101010008FFF34462846FFF76BF8641EFAD2F6E7D6
:101020006D1200006164632076616C7565206973E0
:101030000000000008610000F8B504465920524D38
:101040001622882128602A6029602B68002BF9D09D
:101050004E48FFF7DDF84E48FFF7DAF8FFF70AFCD5
:1010600000232B6005221207906B4A4908409063C9
:10107000916B012080020143916347498D680926E5
:1010800035438D60956B454E35409563956B4600B5
:10109000354395638D68902635438D60956B404E42
:1010A00035409563956B8600354395638D680926B9
:1010B000360235438D60956B3A4E35409563956B9E
:1010C000C600354395638A6809252D032A438A6043
:1010D0000D68FF2212029543260235430D604D68CC
:1010E00007273F02BD432818486088684000400831
:1010F0008860CB627D20C00048610D682D0A2D02FA
:1011000025430D604D687027BD4340354D608D68A7
:101110006D006D088D608B6208610D682D0A2D02CF
:1011200025430D604C68E408E400241D4C608C6885
:10113000640064088C604B62C8600C68944334435C
:101140000C604A683C02A2430124A40312194A60BD
:101150008A68520052088A600B638861886801229D
:1011600010438860886810221043886088688A1558
:101170001043886088681201104388604B628B625C
:10118000CB620B63F8BD0000000100501400C0A743
:101190001500E0A7FBFBFFFF00000440F7F7FFFF8F
:1011A000EFEFFFFFDFDFFFFF1CB508A00068019035
:1011B00000F00EF82C2000900D231422032101A82A
:1011C00000F0A2F900F030FA1CBD00002323230038
:1011D000F8B505242407206B2063206B07256D03D9
:1011E00028432063134841684160134E3046FFF79F
:1011F0000FF8012210213046FFF7BCF9012202212D
:101200000E48FFF70FFA002204210D48FFF70AFAF3
:10121000206B284320630B480B4C009008230422CA
:1012200000212046FFF751FA2046FFF749FA002037
:101230002062F8BD400000500C0040A60040005065
:101240004041005080841E000000034006490862AF
:1012500008680122104308600868C043C007FBD03B
:101260000869C0B270470000000003401CB5064981
:10127000022048800020009001901223034A102190
:101280007620FFF791FE1CBD1400002070000020A6
:1012900010B50446016810A0FFF724FC11A0616896
:1012A000FFF720FC12A0A168FFF71CFC13A0E16867
:1012B000FFF718FC14A02169FFF714FC15A0616961
:1012C000FFF710FC16A0A169FFF70CFC17A0E1695D
:1012D000FFF708FC10BD0000723020203D20307860
:1012E00025780A00723120203D20307825780A00C8
:1012F000723220203D20307825780A007233202079
:101300003D20307825780A00723132203D20307837
:1013100025780A006C7220203D20307825780A005C
:10132000706320203D20307825780A007073722089
:101330003D20307825780A0010B51AC91AC00C383B
:10134000511C00D0826010BDF8B58C460546500196
:10135000990041181348069F0918079E29607C01CF
:10136000B100611808186860012460462146994060
:10137000A8609001A20310430522120780180222E0
:10138000FFF750F9B4400122B8019203104305223F
:101390001207801821460222FFF744F92846FFF77A
:1013A0001EFCF8BD00420050FFB581B01F460E463E
:1013B0000546002472B6FFF7FCFB7600F1B2284622
:1013C000FFF71BFC2846FFF7BEFB002832D128465A
:1013D0000399FFF712FC2846FFF7B5FB002829D137
:1013E0002846FFF7E6FB761CF1B22846FFF705FC1E
:1013F0002846FFF7A8FB00281CD10A9E761E0CE0A9
:10140000FFF7B9FB38552968002008602846FFF728
:1014100088FB296801200860641CB4422846EFD389
:10142000FFF7A9FB38552968012008602846641C8D
:10143000FFF777FB2846FFF7D2FB62B6204605B0E0
:10144000F0BD000070B504460D460F48FEF7E0FE03
:1014500022460E4C0121C9062046FFF787FA002DCF
:101460000AD02068610308432060481508490860D5
:1014700002210820FFF702F90648056020680121D3
:1014800089070843206070BD020080AE0000014063
:1014900000E100E06000002010B50D48FEF7B8FE46
:1014A0000D490C4848600D4841680122520491439F
:1014B00041600B4CE12149022046FFF7D3FA6068F6
:1014C000112108436060012006490003086010BD37
:1014D000103D80A703030000400000504041005031
:1014E0000000054000E100E010B50021E12000F01F
:1014F000BBF80021E22000F0B7F810BD10B5702154
:10150000272000F0B1F810BDFFB50D463EA003C87E
:1015100087B0019100903EA000683EA1049003C9ED
:10152000039102903DA0006805903DA000680690E0
:101530001E465A21532000F097F8A521532000F0B1
:1015400093F80124374F02E03846FEF7D1FD641EC0
:10155000FAD2FFF7C9FFFFF7D1FF212E01D20021F8
:1015600000E018213D2000F07FF80021FD2000F070
:101570007BF80321222000F077F8A81EC1B22320B7
:1015800000F072F82520099900F06EF831463120FC
:1015900000F06AF83146322000F066F82A46302022
:1015A000079900F04BF82A462A20079900F046F8E0
:1015B000052269463F2000F041F8062202A93A20A0
:1015C00000F03CF8012205A9392000F037F8032289
:1015D00004A93E2000F032F8032206A93B2000F0C7
:1015E0002DF800213C2000F03FF82620109900F053
:1015F0003BF80021242000F037F80021212000F0E2
:1016000033F80BB0F0BD000012ED679C46000000FF
:10161000F63F5D004521EF2C5A400000010000001C
:101620000BDF02000861000010B58F21202000F0C0
:101630001BF80021FD2000F017F810BDF8B50F468B
:10164000084E002115467160FFF700FE002404E0FB
:10165000385DFFF7FBFD641CE4B2AC42F8D3012017
:101660007060F8BD0042005070B50D46054C002179
:101670006160FFF7EBFD2846FFF7E8FD01206060A1
:1016800070BD000000420050A816000000000020BD
:1016900070000000040B000018170000700000200C
:1016A00098020000140B00000080510100805101DD
:1016B000000000000000000000000000000000002A
:1016C0001232440000000000000000000000000092
:1016D0006400900158022003121212121212121208
:1016E00013121212131212121212121212131212D7
:1016F00012131212121212121212131212121312C7
:1017000000000000000000000000000000000000D9
:081710000000000000000000D1
:04000005000000F9FE
:00000001FF
